:020000020000FC
:100000005CCEB7C10000000020C0000089C0000025
:10001000000093C00000000000000000020304067E
:10002000080C10182030406080000406080C1018DE
:100030002030406080A0C0000003070F1F000D0D9E
:100040000403060D0502030202004FB662FD0CC058
:10005000552041F00994C52DC095089483FDC7959E
:10006000C4BD64604FBE1895C0916400089483FDC0
:10007000C795C4BD6B7FC0916400CF3F09F419C020
:100080004FBE9098919893981895909891989398BE
:1000900076FD0DC065FD0BC0C9E0CA95F1F7C091B2
:1000A000B100C0FD959AC1FD979AC2FD949A4FBECA
:1000B000189524BCCC27C064C8BF6460F8CFCBCFF0
:1000C00070FFC9CF65FDC7CF909AC5CF70FFC3CF72
:1000D00065FDC1CF919ABFCF70FFBDCF65FDBBCF8E
:1000E000939AB9CF959870FFB6CF65FDB4CFCEE1A6
:1000F000CA95F1F7909AAFCF979870FFACCF65FD96
:10010000AACFCEE1CA95F1F7919AA5CF949870FF46
:10011000A2CF65FDA0CFCEE1CA95F1F7939A9BCF10
:100120004FB6C9B7CF7EC9BF6E7FCCB5CE0DDDB59A
:10013000DF1DDBBDCABD4FBE18953FB68F7EABB786
:10014000A074A2118061A0E0ABBFA9B7AE7FA9BF28
:100150007894A0916800AA2341F085FD2AC0A0915F
:100160006800AA95A093680024C040E050E085FD97
:1001700014C0A0B396FDA095A2FD4FEFA3E096FD9D
:10018000A2E0A5BFAA27A064AABF8D7FA0B396FD59
:10019000A095A2FD5FEF451741F7A0E461FDA09394
:1001A000680085FD03C0A0E4A0936800409396001A
:1001B000816085FD0EC0A0916900AA2331F0A09155
:1001C0006900AA95A093690004C08061AA27A06471
:1001D000AABF80FF0AC0A09196004A2F61FF8E7FC0
:1001E00085FD01C000C0409361004091B4004430DF
:1001F00009F004C0A0916100A0936300A52DA03474
:1002000008F06860A0916000A395A093600051F091
:10021000F894A9B7A160A9BF84FF02C0A0E4ABBF56
:100220003FBE1895A0917400A395A093740042E07E
:1002300050916800552329F085FF03C05A955093CB
:100240006800A0919600A13018F0209299000DC08E
:1002500020929A002092A300A0919900AF5FA093F2
:10026000990018F0AFEFA0939900B0906100509101
:10027000B400523049F466FF91F0A2E3BA1678F068
:10028000A0918600A0936100533049F466FF39F0D5
:10029000A2E3BA1620F0A091C000A0936100509193
:1002A00062005B1521F010F05A9501C053955093F0
:1002B00062004A95D1F65091A300539509F45A95DE
:1002C0005093A300A091A400AA95A093A40009F0C4
:1002D00046C0A1E0A093A40045E0A091A5005A1754
:1002E000F0F1A091A6005A1728F441E0A3E0A093F2
:1002F000A40007C0A091A7005A1718F441E040934A
:10030000A400D0909C00C0906300DC14A8F0A091E1
:10031000B400A430D9F066FD0FC0C0929C00539584
:1003200011F0A091A500A093A300A1E0A093A400C8
:10033000ACE3A093620013C0A0919C00A40F20F432
:100340005FEF50939C0002C0A0939C00A0919C0082
:10035000AF3F29F4AFEFA0939A00A093A300F894C5
:10036000A9B7A160A9BF84FF02C0A0E4ABBF3FBE94
:1003700018953FB64CB55DB58F7EABB7A074A21192
:100380008061A0E0ABBFA9B7AE7FA9BF789481FD23
:1003900023C0A2E096FDA3E0A5BF8260A0B396FDB6
:1003A000A095A2FF05C040936500509366001CC154
:1003B000A3E096FDA2E0A5BFAA27A064AABF8D7FF7
:1003C00085FF01C004C140E0A0B396FDA095A2FD49
:1003D000FEC040939600EDC0A3E096FDA2E0A5BF4D
:1003E0008D7F61FF71C0A2E096FDA3E0A5BFAA27A3
:1003F000A064AABF82604093910050939200A090A5
:100400008F004A19B09090005B09BB24A22C4C3895
:10041000520518F42092950049C0A091D400AA2357
:1004200059F1483C520528F4A0E1BA2EAAE0AA2EC0
:1004300023C04836A1E05A0728F4A8E0BA2EAFE05E
:10044000AA2E1AC0403DA2E05A0728F4A4E0BA2E12
:10045000AEE1AA2E11C0403AA5E05A0728F4A2E066
:10046000BA2EACE3AA2E08C04839A8E05A0720F4F7
:10047000A1E0BA2EA8E7AA2EC42EA0919300CA1A12
:10048000D52EA0919400DA0ADD202AF4AFEFC094B3
:10049000D094CA1ADA0A20929500A8E0A210A0E02F
:1004A000CA14DA0618F4A1E0A093950040939300D3
:1004B00050939400409191005091920040938F008E
:1004C0005093900042E075C0A09165004A1BA09136
:1004D00066005A0B94FD60C093FD5EC092FD5AC049
:1004E00086FF03C0D52EC42E0CC05695479591FDAE
:1004F00051C05695479590FD4DC0D52EC42ED6942B
:10050000C79461FD19C0AC2DAC51AD2DA24008F0CF
:1005100005C0DD2089F4AC2DA85C70F4A0916700C3
:10052000A395AA2311F0A0936700AA3008F44FC046
:100530002092960081604BC0A0916700AA2319F019
:10054000AA95A0936700A22C5091BA0097FD02C013
:10055000A090C800AAEFAA0EA22DA21DCA18DA0AFE
:100560004FB74170442319F040E050E015C0AFEFA1
:10057000CA16D20418F04FEF50E00EC0A091AC00A4
:10058000CA9E412D000C441F50E008F012C04FEFEE
:1005900050E00FC05695479594FF07C0552309F0CA
:1005A0004FEFA42FA6954A0F521D4F3F520508F05A
:1005B0004FEF40939600816061FF09C0AFE1A095C5
:1005C000A923AB299A2F8F7DBB2009F48062A0E478
:1005D000A093680085FF03C0AAE0A093680061FDB6
:1005E00003C085FD01C08F7E85FD03C0A0E2A093FE
:1005F0006900F894A9B7A160A9BF84FF02C0A0E474
:10060000ABBF3FBE189511E00AC013E008C01AE066
:1006100006C01EE104C014E602C018EC00C005E1EB
:10062000BB27BA95F1F70A95D9F71A95C1F708953E
:100630002AE338E709C020E33CE806C02AE234EBAD
:1006400003C025E238EC00C012E0BB279798BA95AA
:10065000F1F7919ABA95F1F79198BA95F1F7979ABF
:10066000BA95F1F7123009F0909A123009F4939A82
:10067000B091AD00BA95F1F7123009F090981230B0
:1006800009F49398B7E8BA95F1F71A95F1F6022FA5
:10069000B22FBA95F1F70A95D9F73A95A9F6979836
:1006A0000895221B39E0001F3A9509F40895221F8E
:1006B000211B18F4210F8894F6CF0894F4CF622CF4
:1006C000722CB0E08894B395221F331FE0F7379562
:1006D00027958894912E802E020B130B10F4192D60
:1006E000082D10F4889401C00894661C771CBA95F4
:1006F00071F7172D062D0895322D11232AF43A95FE
:1007000000951095031B130BF894029F712C002D7C
:10071000129F912C802C7894780C172D921C292DE7
:10072000B4E06B2E2695179507956A94D9F7332375
:1007300021F000951095031B130B08950091B40050
:10074000043009F474C0B0919600B95198F0B72FF5
:10075000B67081F466FD2BC005E09090C600B92DFF
:10076000BA9521F00AE0BA9509F002E1B0917B0058
:10077000B01BE0F066FF0AC0B0919E00B0939C00F1
:10078000BFEFB093A300B1E0B093A400B0916100BB
:10079000B093630020927E0020927F002092800020
:1007A00020928100209282006F7B41C06064909013
:1007B000C600B92DBA9579F4B0916200B095BB1F0F
:1007C000BB1F1B2FB7950B2FB12FB170B3951B2FEC
:1007D000B02FBE7F25C0B92DBA95BA9581F4B091DE
:1007E0006200B095BB1FBB1FBB1F1B2FB7950B2F04
:1007F000B12FB370B3951B2FB02FBC7F14C0B09135
:100800006200B095BB1FBB1FBB1FBB1F1B2FB79543
:100810000B2FB12FB770B395B3951B2FB02FB87FA7
:10082000B0540B2F120900937E0010937F0008959F
:1008300010917B00169500917A000795B0917E008B
:10084000B01B0B2FB0917F00B10B1B2F28F4003889
:10085000BFEF1B0740F009C00F37120508F405C0B1
:100860000FE710E002C000E81FEF00938300109331
:100870008400089500918300B09180000B0F1091C7
:100880008400B09181001B1F20E03091840033234D
:100890000AF42A95B09182002B1F1AF4203F40F0F1
:1008A0000AC02F3008F407C00FEF1FEF2FE003C07E
:1008B00000E010E020EF30916300B0919B003B1707
:1008C00018F4323030F009C0B0918400BB235AF0E4
:1008D00004C0B0918400BB2332F4009380001093D5
:1008E00081002093820008952091D7000091830019
:1008F000000F10918400111FFFDE11232AF400382D
:10090000BFEF1B0740F009C00F37120508F405C000
:100910000FE710E002C000E81FEF002352F0B09193
:100920006200B01B0B2F18F0013008F00AC001E084
:1009300008C000950F5FB09162000B0F08F001C076
:100940000FEF0093850008952091D8000091810059
:1009500010918200D1DE11232AF40130BFEF1B0772
:1009600040F009C00F3F120508F405C00FEF10E07A
:1009700002C001E01FEF112352F0B0918500B01BBF
:100980000B2F18F0013008F00AC001E008C00095F4
:100990000F5FB09185000B0F08F001C00FEF0093BF
:1009A000630008950FEF677F71FD29C072FD09C0D4
:1009B0006860B0917B00BA3020F0B52DB03408F4F7
:1009C000677FB091D300BB23D1F0B0917B00BB23F4
:1009D000B1F00FEF10917B0064DEF894B0917300DA
:1009E00072FDB5E00B9F112D002D7894112309F0B5
:1009F0000FEFB0919E000B1710F400919E00009332
:100A00009D00089500917A0010917B0000541140E0
:100A1000B0919D0010F4BA9501C0B39511F0B09358
:100A20009D000895E7D3B7E074FDB7E0B06CB7B9A7
:100A3000B6B1B068B064B6B9E6DDB7E074FDB7E052
:100A4000B06CB7B9B6B1B068B064B6B9B6B1B6FDFE
:100A5000FDCF04B115B1B6B1BF77B6B922D425E642
:100A60002093A800222309F441C030E03093A9006C
:100A7000732E7694622E6694620E731E262D372D89
:100A80000217130778F08090A800B5E6B80DB09370
:100A9000A8008090A900B0E0B81DB093A900260D71
:100AA000371DEECF8090A8009090A9001091A9006A
:100AB00016950091A80007951695079523E01695C1
:100AC00007952A95E1F72091B5002A9529F42092FF
:100AD000A8002092A9000AC02A9521F0800E911E3C
:100AE0002A95E1F78092A8009092A900089520919C
:100AF000B500B6B1B6FDFBCF04B115B1B6B1BF7745
:100B0000B6B9B091AA00B395B093AA00B83060F11D
:100B10002092AA00B091D200BB2321F1112329F029
:100B2000B091AB00BF3F61F009C0B091AB000B17B3
:100B300039F020F4BB2321F0BA9502C0B395E1F35C
:100B400000919B00B093AB00B03050F400ECB0309B
:100B500038F400E8B03020F400E4B03008F400E0ED
:100B600000939B007F7E08952130B1F00F3FB3E0EA
:100B70001B0790F4B5E6BB2379F0B091A8000B17E2
:100B8000B091A9001B0740F4B0919B00BB2359F022
:100B9000BA95B0939B0007C0B0919B00BF3F19F07E
:100BA000B395B0939B0000919B00B0916300B01B84
:100BB00010F400916300B0919C000B1750F000916D
:100BC0009C00B0919C00BF3F21F0B0919C00B0937D
:100BD0009B00502E00936400B091AA00B73009F436
:100BE0007061089502E3F894B091D9000B9F012D34
:100BF000000C001F7894B0919B000B1710F000912F
:100C00009B000093610000936300502E00936400EA
:100C100000939E00089520927A00B0EFB0937B007D
:100C20000895F8940CB51DB5209174007894309116
:100C30007500609076000093750010937600031B9A
:100C4000160971FD03C077FD7DC027C07090770045
:100C5000209377002709222311F00FEF1FEF8090D8
:100C6000780090907900309378006092790000913C
:100C70007500109176000819190920917A003091B9
:100C80007B0036952795020F131F10F40FEF1FEF0F
:100C900000937A0010937B0029C020917A00309154
:100CA0007B003901B4E08B2EB2E09B2E343010F083
:100CB0008A949A94383010F08A949A94769467942F
:100CC0008A94E1F726193709992021F0169507959E
:100CD0009A94E1F7200F311F20937A0030937B0024
:100CE00028F43FEF30937A0030937B00323008F4E1
:100CF000706871FF02C0B3E00DC0B091C4000091F4
:100D00007100023838F0B395003A08F0B395B63068
:100D100008F0B5E09B2EB4E08B2E10917B00009183
:100D20007A0024E0169507952A95E1F7081912092B
:100D300028F0B02FB250B12FB20910F402E010E049
:100D4000980126C020917A0030917B003901769479
:100D500067946694669466942619320906950695FA
:100D6000200F321D20937A0030937B00323008F040
:100D70007F7704E036952795369527952695269515
:100D8000201B10F0223008F422E089019090C4006A
:100D900060FDFECFE0908B00F0908C006160B9B7F1
:100DA000B061B9BF380177FD41C076946794009374
:100DB0008B0010938C00B92DB330E1F0B0FD04C06E
:100DC000060D171D930106C0000F111F02501209D6
:100DD00022E030E0B92DB33068F020938D003093DD
:100DE0008E000093870010938800609289007092B3
:100DF0008A003AC000938D0010938E0020938700E4
:100E0000309388006092890070928A0071FF0DC053
:100E1000BFE0B0938D0020928E00B09389002092A5
:100E20008A00B0938B0020928C001EC066940093C1
:100E30008B00B92DB33091F0B0FD03C0060D262D07
:100E400003C0000F025022E0B92DB33038F02093D8
:100E50008D00009387006092890006C000938D008A
:100E6000209387006092890000917C0002FD03506E
:100E7000013031F495FD0CC0B2E0B06CB7B90BC0D5
:100E8000023021F4B3E0B06CB7B905C095FDF4CFE2
:100E9000B4E0B06CB7B90091A200000F10F4BBE64B
:100EA0000B270093A20060FDFECFB2E0B0936E006E
:100EB0006160B9B7B061B9BFB72FB670D1F02091FA
:100EC0007A0030917B00369527953695279571FFEE
:100ED00002C0B0E43B0FF8940CB51DB5020F131F10
:100EE0001BBD0ABD6160B0E1B8BFB9B7B061B9BFA1
:100EF00078940895606120927D0020E067FD20E2F3
:100F000006C0606120927D0020E267FD20E001E0E4
:100F100011E077FD11C0B72FB67009F06F7E14E1B4
:100F200000917B00069509F403950F3008F00FE05F
:100F300071FF02C004E114E160FD0FC0B0917D00BB
:100F4000BB2359F071FF06C0B0916E00BA95B09303
:100F50006E0011F4706247C0ABDFB0B7B77FB0BFAF
:100F6000B8B1B0B7B860B0BFB0917D00B395B093E1
:100F70007D00B8B177FD06C0B1E071FDB3E0BA9570
:100F8000F1F7B8B1B072B21709F022C071FF05C015
:100F90000395011708F00A95CFCF64FD05C00395AE
:100FA000011708F0B4CFC8CF6F7EF8943CB56DB48C
:100FB00070907A0080907B00370D681C6BBC3ABD46
:100FC0006160B0E1B8BFB9B7B061B9BF78949FCFE5
:100FD000B0916D00B13008F49ACF64FD98CF0A95B6
:100FE00009F0AACF7F7D20918D0030918E00F8947A
:100FF000B0E1B8BF0CB51DB5020F131F1BBD0ABD74
:10100000E0908700F09088006160B9B7B061B9BF27
:101010007894B72FB67039F0B0916D0072FFB39528
:10102000B0936D0009C075FF07C067FD05C064FD82
:1010300003C0BF91BF91E8C4089500E063FF03C0FF
:1010400064FF01C001E0F89410917100B7E01B9FAC
:10105000212D102D7894200F2695179526951795FC
:101060002695179510937100183718F4B8E7B093C8
:10107000710000917100B09172000B1720F0606256
:1010800090989198939860FDFECFE0908900F09041
:101090008A006160B9B7B061B9BF0895B2E095FD4B
:1010A0000AC0F894B0937C009798959A62FF01C0AB
:1010B000939A7894F4C0F894B0937C009798949A9B
:1010C00062FF01C0909A7894EAC0B3E082FF24C026
:1010D00095FD11C002E0F894B0937C00ECE7F0E0DD
:1010E0000093B1009398949862FF02C0919A01C056
:1010F000979A7894D4C002E0F894B0937C00ECE71F
:10110000F0E00093B1009098959862FF02C0919A28
:1011100001C0979A7894C3C095FD0BC0F894B09322
:101120007C00E6E6F0E0939862FF01C0919A789423
:10113000B6C0F894B0937C00E6E6F0E0909862FFC9
:1011400001C0919A7894ABC0B4E095FD0AC0F894C0
:10115000B0937C009598949A62FF01C0919A78941C
:101160009EC0F894B0937C009498959A62FF01C059
:10117000919A789494C0B5E082FF24C095FD11C087
:1011800001E0F894B0937C00E2E7F0E00093B10056
:101190009198979862FF02C0909A01C0959A7894AE
:1011A0007EC004E0F894B0937C00E6E8F0E00093A1
:1011B000B1009198979862FF02C0939A01C0949AE7
:1011C00078946DC095FD0BC0F894B0937C00E0E678
:1011D000F0E0919862FF01C0909A789460C0F89412
:1011E000B0937C00ECE6F0E0919862FF01C0939A26
:1011F000789455C0B6E095FD0AC0F894B0937C0091
:101200009498979A62FF01C0909A789448C0F89495
:10121000B0937C009598979A62FF01C0939A789456
:101220003EC0B1E082FF24C095FD11C004E0F894F7
:10123000B0937C00E6E8F0E00093B10090989598B8
:1012400062FF02C0939A01C0949A789428C001E08A
:10125000F894B0937C00E2E7F0E00093B10093983B
:10126000949862FF02C0909A01C0959A789417C032
:1012700095FD0BC0F894B0937C00ECE6F0E09098FC
:1012800062FF01C0939A78940AC0F894B0937C00EE
:10129000E0E6F0E0939862FF01C0909A78946F7D49
:1012A00008952FE530E0F9012092B10090989198CF
:1012B00093989598979894986B7F0895A2EBB0E0D7
:1012C00007E00D9307E00D9301E00D9304E00D930B
:1012D0000FEF0D930D930AE00D9302E00D9301E0E3
:1012E0000D9301E00D93AEEBB0E001E00D9300E053
:1012F0000D9304EB0D930FEF0D930D930D9303E0FE
:101300000D930FEF0D9301E00D930FEF0D9305E299
:101310000D9300ED0D9308E70D9308EC0D9304E099
:101320000D930FEF0D9301E00D9300E00D930AE78D
:101330000D930AE00D9300E00D9301E00D9300E0A2
:101340000D930FEF0D9300E00D9308952091B900D8
:101350008B7FB091BA009F7DB1FD90629F7BB09171
:10136000BB00B1FD9064223011F0886001C0877F1E
:1013700008950A95E00FF21DB4910895ECE1F0E0B4
:101380000091B200F6DFB093D700ECE1F0E00091FD
:10139000B300EFDFB093D800EAE2F0E00091B800CC
:1013A000E8DFB093D9000091D100002309F4039540
:1013B000013108F001E1B02FB00FB00FB093A500DC
:1013C0001B2FB10FB10FB00FB093A600B10FB00F2C
:1013D000B00FB093A7000091B800023008F402E00B
:1013E00000937300B091CE000FEFB23009F400EA21
:1013F000B33009F402E800937200E8E3F0E00091F2
:10140000D500B7DFB093A000089508952091C800DB
:101410003091C900B091BA00B33009F43E5097FF43
:1014200002C020E03FEFB32FB21B6B2EB25810F476
:10143000B2E86B2E00E00395609EB12DBD57D8F346
:101440000093AC0008959068E1DFE3D820E030E03D
:10145000B0E16B2EDAD8B09196002B0F321D6A9452
:10146000C9F7B4E036952795BA95E1F7822E9F77B4
:10147000CDDF0895F894E3E0F0E0B9E0B7BFB491B0
:10148000B078C1F3F894A895B1B5B861B1BDB0E03A
:10149000B1BDB4E0BEBFBFE5BDBF03DFB0E0B8BBC8
:1014A000B0E1B7BBB0E0B5BBB0E0B4BBB0E0B2BB3D
:1014B000BBEBB1BB2224A0E0B0E02D92AA31E9F74A
:1014C000A0E6B0E00FEF2D920A95E9F7B1E0B093F6
:1014D000A200F4DEDAD2B7E0B06CB7B9B6B1B4604E
:1014E000B068B6B90091CA000093AD00B1E0B09306
:1014F0006A00F89492D89CD88CD89DD88AD89ED867
:1015000088D852D38AD889D886D8F8940AEF1AEFA7
:10151000A0B396FDA095A2FF1FC01A95C9F70A9522
:10152000B1F7E0E0FCE1B591B43E39F4B591B03EDD
:1015300021F4B591BF3F09F40CC0E0E0F395F395B9
:10154000B591B83F49F4B591B43931F4B591BA3A8F
:1015500019F4EE27F6950994F9DE10DF56DF56DF11
:101560000091CA000093AD009CDEB2E0B3BFB2E0D0
:10157000BEBDB2E0B5BDB1E5B8BFB9BFB0B7B77FCA
:10158000B0BFB8B1B0B7B860B0BF3DD878944ADA50
:1015900020927000B3E096FDB2E0B5BFB0E4BBBFEF
:1015A000BB27B064BABF8D7F38D8626033E02CE0CF
:1015B000B0919500BB2321F42CE03A9509F4A5CF16
:1015C00028D880FFA2CF8E7FB0919600B23078F3FA
:1015D000B92FBF710091980000939700B0939800C5
:1015E000B01729F72A9521F76D7FB3E096FDB2E099
:1015F000B5BFBB27B064BABF8D7FB091D400BB2309
:1016000021F48062B92FB0709B2F8F7B20926700EE
:1016100002D885FF05C0B0916700BA3008F0806439
:10162000F4D702E085FF01C000E0B0919600B0174A
:10163000B8F3F894FDD7FCD7FBD77894EED7209277
:101640008600E3D7B091BE00B13008F46EC0B0910F
:101650006A00B13008F469C085FD18C0B0919600E9
:10166000BF3F08F462C0F894ECD77894D4D7B09117
:101670009600B130C0F7F894DBD7C9D7D9D77894A2
:10168000CAD7B0919600BF3FB0F3C0C2B8E09B2E5E
:101690009068F894BBDE7894BED7F8949F77B6DE56
:1016A00080909600B0919600BF37789408F445C0BA
:1016B000AAD7F894C6D778949A9451F7C4DEB82D77
:1016C000B550B093C900A9D7F8940CD272D27894CF
:1016D000BAE09B2E9068F89499DE78949CD7F894A1
:1016E0009F7794DE80909600B0919600BF377894F3
:1016F00078F789D7F8949CD78AD79AD778949A9410
:1017000049F7A1DEB82DBB5FB093C80086D7F89427
:10171000E9D15ED278947FD7F89478DE7894B0914E
:101720009600BF3F08F498CF71C200919600B09127
:1017300086000B1710F0009386006DD701E0B09182
:10174000BA00B35009F405E0B0919600B01708F064
:1017500078CFF89476D775D774D778945ED72092DF
:101760006A0020926B0020926C00B0916B00B395E0
:10177000B0936B00BF3F71F5B0916C00B395B0931F
:101780006C00B091CC0009E1BA9559F002E3BA952A
:1017900041F00DE7BA9529F00AEFBA9511F02092C1
:1017A0006C00B0916C00B017A8F07BDD2CD7B09125
:1017B0006C00BA95B0936C0020926B00B091CB0096
:1017C000B093AD00F8943DD77894B091CA00B0932F
:1017D000AD0021D71CD7B0916800BB2319F485FF59
:1017E00001C093CE01E085FD01C006E0B0919600F6
:1017F000B01708F4BACF0FD7B0916800BB2309F433
:1018000084CEF8944EDD20926100209262002092F6
:101810006300522C209264002092A1007894B09131
:10182000B700BB0FB0939F0020927E0020927F00F4
:101830002092800020928100209282002092AA00B3
:1018400060E070E020927100B8E0B093AA0070618F
:10185000DAD6B7E074FDB7E0B06CB7B9B6B1B0682E
:10186000B064B6B9B6B1B6FDFDCF04B115B1B6B12D
:10187000BF77B6B9112309F00FEF0093AB0037D94A
:10188000B8E0B093AA00706161DDF894BFEFB09347
:101890009B00A8D9B0916100B0939B00B0939C00CD
:1018A000B0939D007894B1E0B0936100B093630071
:1018B0005B2EB0936400B093A400B0919A00B093F3
:1018C000A300B091BA00B33019F49F7D87FD9062F8
:1018D0007160726020926D008DDCA3DC9CD9A1D96F
:1018E0009AD99FD998D90DDB29D7A7DBD7DB99D90E
:1018F00001DB66FD9DD777FF55D877FD83D89DDB4B
:10190000E4DB8FD9FEDA66FDB5D797DB1DDC89D91C
:10191000F1DA66FDE9D791DB2EDC83D9F2DA66FDD8
:1019200013D88BDB67DC7DD9E5DAB7E074FDB7E06F
:10193000B06CB7B9B6B1B068B064B6B97EDB71DC73
:1019400070D9D5D871FF1EC0B0919E00B0939B0096
:10195000B0939C00B0919A00B093A300B1E0B09313
:10196000A40018E12CE0B0916D00B11728F07D7F44
:10197000746020936F0006C0B0919600B13008F0FB
:10198000B2CF4CC072FF11C067FD0FC0B0916F00A5
:10199000BA9519F47B7F7860A6CFB0936F00B091B1
:1019A0009600B13008F09FCF39C020927000B091FE
:1019B0009900B13058F0B0919E00B0939C00B09166
:1019C0009A00B093A300B1E0B093A400B091990045
:1019D0000AEF1091D600112309F003E0B01708F0C8
:1019E0001DC085FF04C0B0916800BB23B9F000EFB3
:1019F00067FF05C0B0919E00B0939B0000E2B091DC
:101A00007B00B01708F46FCFB0917000B395B0931E
:101A10007000B0919600BB2309F002C020927000C4
:101A2000F8943FDC8090B900B2E0B093B9008EDC4E
:101A30008092B9002092610020926200209263009F
:101A4000522C2092640020929F0060E070E0789415
:101A5000E2D527DC0091D600002319F0909A919AE4
:101A6000939AB7E0B06CB7B9B6B1B460B068B6B924
:101A700085FF05C0B0916800BB2309F446CDB09145
:101A8000BF00B13008F0CCCD6CCEEDE0F0E023D05B
:101A9000053A09F01BC0EEE0F0E01DD00A3509F070
:101AA00015C03AE0A2EBB0E0E3E0F0E014D00D9313
:101AB00031963A95D9F739E1AEEBB0E0EFE0F0E0DE
:101AC0000AD00D9331963A95D9F702C0F7DB0AD0C8
:101AD000E8E2F0E00895E199FECFEEBBFFBBE09AAB
:101AE0000DB308951ED03AE0A2EBB0E0E3E0F0E0E1
:101AF0000D910FD031963A95D9F739E1AEEBB0E0C0
:101B0000EFE0F0E00D9105D031963A95D9F712D07B
:101B10000895E199FECF0DBBEEBBFFBBE29AE19ABF
:101B20000895EDE0F0E00FEFF4DFEEE0F0E00FEF0E
:101B3000F0DF0895EDE0F0E005EAEBDFEEE0F0E045
:101B40000AE5E7DF08953091AE000091AF00313033
:101B500011F40093B200323011F40093B30033302B
:101B600011F40093B400343011F40093C600353002
:101B700011F40093B500363011F40093B8003730FB
:101B800011F40093C400383011F40093B9003930D7
:101B900011F40093CE003A3011F40093BA003B30B8
:101BA00011F40093BB00089525E037D52A95E9F795
:101BB00008953ED540D542D544D529D539D53BD514
:101BC0003DD53FD524D534D536D538D53AD5089529
:101BD00038D534D530D52CD51AD533D52FD52BD5EE
:101BE00027D515D52ED52AD526D522D5089580906E
:101BF000AE009090AF001CD51BD51AD508D58A949D
:101C0000D1F71FD504D59A94E1F70895F894D1DF60
:101C10007894CADFC9DFB1E0B093AE00B1E0B09311
:101C2000AF002092B000F894E2DF7894B5E06B2E1C
:101C300070909600F2D4B09196007B16C9F7B1303F
:101C400018F0BF3F40F107C07EDFF8944BDFB1DFF3
:101C5000B8E0B1BDA9DF6A9459F7B091B000B3956F
:101C6000B093B000B33008F4DECF9EDFB091AF0088
:101C7000B395B093AF00F894B091AE00BA95EEE38F
:101C8000F0E0EB0FF21D049178940395B091AF0052
:101C9000B01708F4C6CF88DF87DFB091AE00B395E8
:101CA000B093AE00B091AE00BC3008F4B7CF06DB05
:0C1CB000F89418DFB8E0B1BD77DFDCCBA2
:00000001FF
